:020000020000FC
:100000000DC0189518951895189518951895189568
:10001000189518951895A4C01895C3C000E00EBF98
:100020000FED0DBF00E808B901E007B906EC06B90D
:1000300004E003BF03E802BF01E009BF4FEE00EF99
:100040000ABB0BBB07E007BBDD27C4E000E3402E83
:10005000502E602E702E70E688277894EE24FF24B0
:1000600020E1359A339A369A45D02223E9F733981E
:100070003598F694E794F694E79402EF11E04AD0AD
:100080001694079416940794A72FBB270D921C92E1
:100090001197EE24FF2420E10D91E00E0D91F01E4A
:1000A0008395803111F4A0E688272A95A9F7129646
:1000B0008395803111F4A0E688277A2F24E0F69406
:1000C000E7942A95E1F733D0A4E0BB27012D0295F0
:1000D0000F70002319F40FEF0D9301C011D0012D03
:1000E00090640ED09F7B002D02950AD0002D08D081
:1000F00001D0B4CF00E205BF8895002705BF089561
:10010000EEEAF1E00F70E00FFB1F049196FD0F7D0A
:100110000D930895222420E11695079510F41E0CE6
:100120002F1C2794179407942A95B1F7089520E17E
:10013000222411240024FF27EE0CFF1C001C111C9C
:10014000221C2A9509F40895E3E002910D5F03FD56
:1001500000830081005D07FD0083E030B1F7ECCF44
:100160000F930FB70F9303E802BF0BB3006F0BBBE6
:10017000C298099138E0C098000F10F4C19A01C0EC
:10018000C198C09A3A95B9F7C29A0BB3006F04238D
:100190000BBB440F10F04FEEC4E00F910FBF0F9157
:1001A000189504B1E00E05B1F01E2A95189530F3AC
:0801B0002AA2E1A424F220A020
:00000001FF
